:020000040000FA
:10000000142160308F0000309000FF308500FF30F9
:100010008600F0308700FE3088000F3089008101B3
:100020001C21880189011021850186018701880131
:1000300089010121D120A0010509A700031D201479
:100040000609A800031D20140709F039A900031DA3
:1000500020140809FE39AA00031D201409090F39CC
:10006000AB00031D201420183828071063001B283C
:100070003A201B28F820A0010509031D20140609B9
:10008000031D20140709F039031D20140809FE3947
:10009000031D201409090F39031D2014201C08001A
:1000A0000714E420A120EF208620EF2027087020ED
:1000B00027087B202808702028087B20290870202A
:1000C00029087B202A0870202A087B202B08702012
:1000D0002B087B202C0870202C087B20DD200800BA
:1000E000A6000830A300A60C03189520031C8F203F
:1000F000A30B73280800A6000830A300A60D031860
:100100008F20031C9520A30B7E2808000C30A20032
:1001100087149B2087109B20A20B88280800871437
:100120009B209B2087109B20080087149B20871012
:100130009B209B2008002830A1006400A10B9D2873
:1001400008008030A4001F30A500BB20AE30A40002
:100150001030A500BB209830A400F030A500BB20D3
:10016000C430A4000030A500BB208230A400393088
:10017000A500BB20080007111030A000A41BCA2056
:10018000A41FC820A50DA40DA00BBE2807150800AC
:100190000810CB28081464008715640087116400D8
:1001A00008000714DD20A1200A21DD200A21DD201E
:1001B000A1200A21DD20071008008230A4000130B0
:1001C000A500BB2087140800003018218D001C21D9
:1001D0008C130C1418210C081021AC0008000230FC
:1001E000A100A2016400A20BF228A10BF4280800D0
:1001F0000A30A100A2016400A20BFB28A10BFD287C
:1002000008006430A100A2016400A20B0429A10B24
:10021000062908000A30A0000121A00B0C290800C3
:100220008313031383120800831303138316080038
:100230008317031783120800831703178316080018
:02400E00CC23C1
:024010000006A8
:00000001FF
